:1000000000308A00B8280000831A0A28A500030ED1
:10001000A6000F288312A500030EA600A6140A0846
:10002000AD008A018313A50E0408A7002008A800CC
:100030002108A9002208AA002308AB002408AC006C
:1000400083128B1E25280B194F28270884002808A7
:10005000A0002908A1002A08A2002B08A3002C0850
:10006000A4002D088A00260E83008312250EA618F0
:10007000831609004108A1014002031842284008E4
:10008000A0004E28A0010830C200C00DA00D4108FC
:1000900020020318A000A10DC20B45285F280630DE
:1000A000810036083502031858283408850059287D
:1000B0008501B50A3508C0000930C1003A2820087A
:1000C000B5000B118A1125283B083D068039BF0079
:1000D000BB1F6F28BA09BB09BA0A0319BB0ABD1FA7
:1000E0007628BC09BD09BC0A0319BD0AA101A201F9
:1000F000A001A3013D08031D80283C0803199A288C
:100100001030BE000310BA0DBB0DA00DA30D3D08AD
:100110002302031D8D283C082002031C96283C085E
:10012000A002031CA3033D08A3020314A10DA20D0A
:10013000BE0B82280000BF1FA228A109A209A10AA4
:100140000319A20A00341030A000A301BE01BB0CA9
:10015000BA0C031CB1283C08A3070318BE0A3D08CB
:10016000BE07BE0CA30CA20CA10CA00BA728E4296F
:1001700084011F3083051F1383161F149F141F153E
:100180009F15073083129F00703083168F00073051
:10019000831299008316050806308312A000A00B75
:1001A000CF28000019088C11831605118312051140
:1001B0000C30950083160108C039023881000030E8
:1001C0008312A10005389200FF308316920083123B
:1001D0008B16C0308B040630810008306500B601F4
:1001E0003608B500AF01AE01B101B001B701370863
:1001F0001D3C031C0629851D04294230A000A00BCC
:10020000FF280000B70A0529B701F7288519062934
:100210008B12B301B201851918290330A000A00B7D
:100220000F29000000000130B2070318B30A0B29A0
:10023000851D25290330A000A00B1C29000000000B
:100240000130B2070318B30A18298B16851D262919
:10025000851928298B12B101B00185193A2903307B
:10026000A000A00B3129000000000130B0070318E6
:10027000B10A2D29851D47290330A000A00B3E2976
:10028000000000000130B0070318B10A3A298B16AC
:10029000851D482985194A29B31B5529B308031D13
:1002A000582932086A3C031C5829B3016B30B2004C
:1002B000B31B6429B308031D61293208C53C031828
:1002C0006429B301C530B2006430B2020030031CAF
:1002D0000130B302B31B7329B308031D93293208FD
:1002E0002E3C031C93290330B40034303202A000AA
:1002F0003308A3000030031C0130A3022008003C97
:10030000B800B9012308031C230FB9023908BB0048
:100310003808BA00BD010530BC0064202208B300D3
:100320002108B200B729B31BB429B308031D9C29C7
:100330003208393C0318B4293030B400343032026A
:10034000B8003308B9000030031C0130B902390885
:10035000BB003808BA00BD010530BC00642022088B
:10036000B3002108B200B7298501B301B2013208F8
:10037000B600B11BC229B108031DC52930086D3C68
:10038000031CC529B101B001E829B11BD329B1086B
:10039000031DCE293008BE3C0318D3290330B10019
:1003A000FF30B000E82964303002B8003108B900ED
:1003B0000030031C0130B9023908BB003808BA000C
:1003C000BD010A30BC00A3282208B1002108B000FA
:1003D0003108A2003008A100A20CA10CA20CA10CB3
:1003E000A20C21089300A20C220C3039A0001508A1
:0A03F000CF3920049500F6286300C1
:02400E00C43CB0
:00000001FF
